:020000040000FA
:1000000000308B000030850000308600031383161B
:10001000C530810010308500F03086008312073033
:100020009F008515051485140A30A800A900A601B3
:10003000A701A001A6116F208D207820A320EF201A
:10004000212134202D2034202D202D20AF0DAF1E56
:100050001B28AF0103102F141B28DF30A300000062
:100060000000A30B2F28080003308A00200800237B
:100070008A01AA000830A4000511AA0D6920031CFA
:100080000515632005156920A40B3C28051169207E
:10009000A71E051563200515692005116920A71EF7
:1000A00005156320051569202108AA000830A40061
:1000B0000511AA0D6920031C05156320051569208B
:1000C000A40B582808002130A3000000A30B6528CA
:1000D00008000430A3000000A30B6B2808002808C8
:1000E000860005100514290886008510851408006F
:1000F0008601851106088515B200AD01321AAD15CD
:10010000B21A2D15321BAD14B21B2D142D08AE00E2
:1001100001302E020319AE010800AB010430AC001F
:1001200086010314860D0310061AA228AB0A861A4C
:10013000A228AB0A061BA228AB0A861BA228AB0A80
:10014000AC0B922808002B1AEB280A302B0203185C
:10015000BD28261908002618B5282614A6142B0831
:10016000A8000A30A90035210800A61808002610AA
:100170002B08A900261524210800A619EC28A6158D
:100180000B302B02031DC8280130AE00A706EC2857
:100190000A302B02031DCF282030A706EC280C3094
:1001A0002B02031DD6280230A706EC280D302B02A7
:1001B000031DDD280430A706EC280E302B02031D9A
:1001C000E4280830A706EC280F302B02031DEC288A
:1001D0001030A706EC28A611A61026110800A61DAF
:1001E000F8280B302B02031DF828C030A1000800AE
:1001F000B00103102F1C0029271C00291030B0006B
:10020000AF1C06292030A7186030B0002F1D0C2924
:10021000303027197030B000AF1D12294030A719B7
:100220008030B0002F1E18295030271A9030B000AF
:100230002E08B00702308A00300800228A01A1008F
:100240000800051A212908002808B1000310310D03
:10025000B10EB10C31072907A000831620089B00BE
:100260001C141A08A7008312080000008316200837
:100270009B0027089A008B131C129C111C155530EB
:100280009D00AA309D009C141C1183120800831647
:080290009C18482983120800A4
:100400008207113491343134B13419349934393488
:10041000B934123492343234B2341A349A343A340D
:10042000BA344534C5346534E5344D34CD346D3497
:10043000ED344634C6346634E6344E34CE346E344D
:10044000EE345034D0347034E4345834D834783402
:10045000F8345234D2347234F2345A34DA347A34CE
:10046000FA34043484342434A4344C348C342C349E
:10047000AC34063486342634A6340E348E342E340E
:10048000AE34143494343434B4341C349C346C346A
:10049000BC34163496343634B6341E349E343E346E
:1004A000BE345434D4347434F4345C34DC347C34AA
:1004B000EC345634D6347634F6345E34DE347E345E
:1004C000FE345134D1347134F1345934D93479345F
:1004D000F9345334D3347334B3345B34DB347B3486
:1004E000FB34053485342534A5340D348D342D3456
:1004F000AD34073487342734A7341B348F342F347A
:10050000AF34153495343534B5341D349D343D3411
:10051000BD34173497343734B7341F349F343B34E9
:10052000BF345534D5347534F5345D34DD347D3421
:10053000FD345734D7347734F7345F34DF347F34C5
:02054000BB34CA
:100600008207AA34C03480343034F034B03420341B
:10061000E034A0340C34CC348C343C34FC34BC3462
:100620002C34EC34AC340834C83488343834F834DE
:10063000B8342834E834A8340334C334833433342E
:10064000F334B3342334E334A3340F34CF348F344E
:100650003F34FF34BF342F34EF34AF340B34CB345A
:100660008B343B34FB34BB342B34EB34AB340234AB
:10067000C23482343234F234B2342234E234A2341A
:100680000E34CE348E343E34FE34BE342E34EE344A
:10069000AE340A34CA348A343A34FA34BA342A3496
:1006A000EA34003440346034973470344834683469
:1006B0005834783444346434543474344C346C34A2
:1006C0005C347C3442346234523472344A346A3496
:1006D0005A347A3446346634563476344E346E3472
:0206E0005E3486
:02400E00293F48
:1042000000000000000000000000000000000000AE
:10421000000000000000000000000000000000009E
:10422000000000000000000000000000000000008E
:10423000000000000000000000000000000000007E
:10424000000000000000000000000000000000006E
:10425000000000000000000000000000000000005E
:10426000000000000000000000000000000000004E
:10427000000000000000000000000000000000003E
:10428000000000000000000000000000000000002E
:10429000000000000000000000000000000000001E
:1042A000000000000000000000000000000000000E
:1042B00000000000000000000000000000000000FE
:1042C00000000000000000000000000000000000EE
:1042D00000000000000000000000000000000000DE
:1042E00000000000000000000000000000000000CE
:1042F00000000000000000000000000000000000BE
:00000001FF
